:020000040000FA
:04000000CD303A289D
:08000800A000030EA100831209
:100010008B1C32288B1031181428B11C3228643004
:10002000010203183128182800001628172818285C
:1000300019281A281B281C281D281E281F283110A3
:10004000B114A810031005190314AA0DA90DA80DC9
:10005000B00B322831152A08AF002908AE00280855
:10006000AD00B11081010B11210E8300A00E200EF6
:02007000090085
:0C007400203084008001840A6030040207
:10008000031C3C281230B000092283160C30850571
:1000900087018312850187010730990000309A009B
:1000A000103083168E008312603083168F00831207
:1000B0000030831691008312C830831681008312AA
:1000C00031309000003083168C00831210308B008A
:1000D000831600309B001C141A088312BC00851D77
:1000E0002323831610309B001C141A088312BD00B2
:1000F000831630309B001C141A088312DE0006237E
:1001000081018E018F010B118B100B108C018B174D
:1001100097203119AD20B30B9528031085190314CE
:10012000B90DF0303902031965216923882864006C
:10013000311808000B1D08000B11B11031141230DA
:10014000B000051DA828321483160113831208007D
:100150003210831601178312080031110130B700E5
:100160008B132030370783169B001C141A08831248
:10017000A400A500C030A5061030370783169B00E9
:100180001C141A088312A3000030370783169B0043
:100190001C141A088312A2008B17321CD5282209BE
:1001A0000339A200A309A409A50922082D02031DF1
:1001B0005F2923082E02031D5F2924082F02031D37
:1001C0005F2901303702031DEA283D18EA283D1453
:1001D0003E14162202303702031DF328BD18F328FF
:1001E000BD143E14252203303702031DFC283D199F
:1001F000FC283D153E14312204303702031D052929
:10020000BD190529BD153E143D2205303702031DD9
:100210000E293D1A0E293D163E144922063037029A
:10022000031D1729BD1A1729BD163E145522073084
:100230003702031D20293D1B20293D173E1464224F
:1002400008303702031D2929BD1B2929BD173E147B
:10025000732209303702031D32295E1832295E14D9
:100260003E147E220A303702031D3B29DE183B294B
:10027000DE143E1489220B303702031D44295E1917
:1002800044295E153E1494220C303702031D4D297B
:10029000DE194D29DE153E149F220D303702031D55
:1002A00056295E1A56295E163E14AA220E303702CF
:1002B000031D5F29DE1A5F29DE163E14B522B70A38
:1002C0000F30370203180800B0280130B600B30021
:1002D000B400B500B70085018701B1139720B30BB7
:1002E000B529031085190314B90DF030390203192B
:1002F000DC29B40BB529013037020319C0220230C2
:1003000037020319C522033037020319CA22043009
:1003100037020319CF22053037020319D4220630E1
:1003200037020319D922073037020319DE220830B9
:1003300037020319E322093037020319E8220A3091
:1003400037020319ED220B3037020319F2220C3069
:1003500037020319F7220D3037020319FC220E3041
:100360003702031901239630B400311D6E29311173
:10037000321CBF292D090339AD00AE09AF092F1C6E
:10038000B1132F1C6E29B11B6E292E186E29B117BF
:100390008B1320303707BB002F08BA00F421103030
:1003A0003707BB002E08BA00F42100303707BB0026
:1003B0002D08BA00F4218B1785018701B70AB60111
:1003C0000F303702031C6E29062308003E1C08006C
:1003D0003E101030BB003D08BA00F4213030BB00A5
:1003E0005E08BA00F42108008B133A0883161C1526
:1003F0009A0083123B0883169B0055309D00AA305B
:100400009D009C1464009C18022A1C1183128B17F7
:100410000800FF30C800CA15CB15CC15CD15CE1578
:10042000CF15D015D115D215D31508008130BD05D3
:10043000FF30DE054130C405C0000030C200C600F8
:10044000BC185F14BC18DF1408008230BD05FF30F3
:10045000DE058030C405C0000030C200C6005F1059
:1004600008008430BD05FF30DE054230C405C00001
:100470004030C200C6005F1008008830BD05FF3064
:10048000DE054630C405C0004030C200C6005F1023
:1004900008009030BD05FF30DE058A30C405C0007D
:1004A0008030C200C6005F100800A030BD05FF30DC
:1004B000DE055130C405C0001030C200C600BC18B3
:1004C0005F14BC18DF140800C030BD05FF30DE0526
:1004D0007130C405C0000030C200C600BC185F14F3
:1004E000BC18DF140800FF30BD05C030DE05403009
:1004F000C505C1000030C300C70008007F30BD053E
:10050000C130DE058030C505C1000030C300C70022
:1005100008007F30BD05C230DE054030C505C10092
:100520004030C300C70008007F30BD05C430DE0581
:100530004030C505C1004030C300C70008007F300F
:10054000BD05C830DE058030C505C1008030C30060
:10055000C70008007F30BD05D030DE054030C5053E
:10056000C1000030C300C70008007F30BD05E03087
:10057000DE054030C505C1000030C300C7000800DB
:1005800010308506003087060800333085060630B7
:1005900087060800203085060030870608002130D5
:1005A0008506003087060800223085060030870661
:1005B00008001030850602308706080010308506D6
:1005C00006308706080000308506103087060800D0
:1005D0000030850608308706080000308506103098
:1005E00087060800003085061030870608000030B6
:1005F000850608308706080000308506103087061B
:100600000800003085061030870608003D181622C5
:10061000BD1825223D193122BD193D223D1A49221E
:10062000BD1A55223D1B6422BD1B73225E187E221B
:10063000DE1889225E199422DE199F225E1AAA22F0
:10064000DE1AB5220800B601B301B4013C1C2B2B05
:10065000BC01BC142D2BBC013C143C08B60064004A
:10066000312B322B332B342B352BFF30B41B850031
:10067000B41F8501B30B2F2BB40B2F2B0310B60C1B
:10068000B608031D2F2B0030BB003C08BA00F42134
:10069000080005125C180516DC1C8512DC1885168E
:1006A0005C1D05105C190514DC1D8510DC19851412
:1006B0005C1E87105C1A8714DC1E0711DC1A0715F4
:1006C0005C1F07105C1B0714DC1F8712DC1B8716DE
:1006D00008008F08031908008F0178308E00C80FBA
:1006E000972DC80A441C992B461C8A2BCA1C7B2BAD
:1006F000CA014A15A72B4A1D802BCA01CA15A72B70
:10070000CA1D852BCA014A16A72B4A1EA72BCA0150
:10071000CA14A72B4A1D8F2BCA014A16A72BCA1D24
:10072000942BCA014A16A72B4A1EA72BCA01CA142A
:10073000A72BCA1C9E2BCA014A15A72B4A1DA32B07
:10074000CA01CA15A72B4A1EA72BCA014A15C41CE9
:10075000CE2BC61CBF2BCB1CB02BCB014B15DC2BDF
:100760004B1DB52BCB01CB15DC2BCB1DBA2BCB01F5
:100770004B16DC2B4B1EDC2BCB01CB14DC2B4B1D87
:10078000C42BCB014B16DC2BCB1DC92BCB014B163D
:10079000DC2B4B1EDC2BCB01CB14DC2BCB1CD32B4B
:1007A000CB014B15DC2B4B1DD82BCB01CB15DC2BF8
:1007B0004B1EDC2BCB014B15441D032C461DF42B8B
:1007C000CC1CE52BCC014C15112C4C1DEA2BCC017B
:1007D000CC15112CCC1DEF2BCC014C16112C4C1E22
:1007E000112CCC01CC14112C4C1DF92BCC014C1626
:1007F000112CCC1DFE2BCC014C16112C4C1E112C97
:10080000CC01CC14112CCC1C082CCC014C15112C77
:100810004C1D0D2CCC01CC15112C4C1E112CCC01D7
:100820004C15C41D392CC61D2A2CCD1C1B2CCD01EA
:100830004D155F13472C4D1D202CCD01CD15472C98
:10084000CD1D252CCD014D16472C4D1E472CCD011D
:10085000CD14472C4D1D2F2CCD014D16472CCD1DF1
:10086000342CCD014D16472C4D1E472CCD01CD14F7
:10087000472CCD1C3E2CCD014D15472C4D1D432C36
:10088000CD01CD15472C4D1E472CCD014D155F1BBD
:10089000702C441E702C461E612CCE1C522CCE0196
:1008A0004E157E2C4E1D572CCE01CE157E2CCE1D06
:1008B0005C2CCE014E167E2C4E1E7E2CCE01CE140C
:1008C0007E2C4E1D662CCE014E167E2CCE1D6B2C22
:1008D000CE014E167E2C4E1E7E2CCE01CE147E2CCA
:1008E000CE1C752CCE014E157E2C4E1D7A2CCE01C1
:1008F000CE157E2C4E1E7E2CCE014E15C41EA52C70
:10090000C61E962CCF1C872CCF014F15B32C4F1D24
:100910008C2CCF01CF15B32CCF1D912CCF014F16AE
:10092000B32C4F1EB32CCF01CF14B32C4F1D9B2CD7
:10093000CF014F16B32CCF1DA02CCF014F16B32CD7
:100940004F1EB32CCF01CF14B32CCF1CAA2CCF0138
:100950004F15B32C4F1DAF2CCF01CF15B32C4F1E0D
:10096000B32CCF014F15441FDA2C461FCB2CD01CC3
:10097000BC2CD0015015E82C501DC12CD001D01535
:10098000E82CD01DC62CD0015016E82C501EE82CA7
:10099000D001D014E82C501DD02CD0015016E82CDA
:1009A000D01DD52CD0015016E82C501EE82CD001BB
:1009B000D014E82CD01CDF2CD0015015E82C501D91
:1009C000E42CD001D015E82C501EE82CD001501595
:1009D000C41F0F2DC61F002DD11CF12CD1015115A4
:1009E0001D2D511DF62CD101D1151D2DD11DFB2C16
:1009F000D10151161D2D511E1D2DD101D1141D2DBA
:100A0000511D052DD10151161D2DD11D0A2DD101CC
:100A100051161D2D511E1D2DD101D1141D2DD11C7E
:100A2000142DD10151151D2D511D192DD101D11597
:100A30001D2D511E1D2DD1015115DF18472D451FAC
:100A4000472D471F382DD21C292DD2015215DF13F7
:100A5000552D521D2E2DD201D215552DD21D332DBF
:100A6000D2015216552D521E552DD201D214552D9C
:100A7000521D3D2DD2015216552DD21D422DD201AF
:100A80005216552D521E552DD201D214552DD21C61
:100A90004C2DD2015215552D521D512DD201D2157A
:100AA000552D521E552DD2015215DF18802DDF1BFA
:100AB000802DC51F802DC71F712DD31C622DD30122
:100AC00053158E2D531D672DD301D3158E2DD31D98
:100AD0006C2DD30153168E2D531E8E2DD301D3149E
:100AE0008E2D531D762DD30153168E2DD31D7B2DA8
:100AF000D30153168E2D531E8E2DD301D3148E2D5C
:100B0000D31C852DD30153158E2D531D8A2DD30152
:100B1000D3158E2D531E8E2DD3015315E62140087B
:100B2000C4004108C5005F18DF145F1CDF104808CF
:100B3000C9000C304A05031D05120C304B05031D7E
:100B400085120C304C05031D05100C304D05031D9E
:100B500085100C304E05031D87100C304F05031D0A
:100B600007110C305005031D07100C305105031DF3
:100B700087120C305205031D07120C305305031D5C
:100B8000871149080E020318F12D12304A05031D82
:100B9000051612304B05031D851612304C05031D3A
:100BA000051412304D05031D851412304E05031D2A
:100BB000871412304F05031D071512305005031D11
:100BC000071412305105031D871612305205031DFC
:100BD000071612305305031D8715FF30480203190D
:100BE00008008F08031D0800972049080E02031C07
:100BF000F12D18304A05031D051206304A05031D64
:100C0000051618304B05031D851206304B05031DD4
:100C1000851618304C05031D051006304C05031DC4
:100C2000051418304D05031D851006304D05031DB4
:100C3000851418304E05031D871006304E05031D20
:100C4000871418304F05031D071106304F05031D8B
:100C5000071518305005031D071006305005031DF9
:100C6000071418305105031D871206305105031D66
:100C7000871618305205031D071206305205031D52
:100C8000071618305305031D871106305305031D41
:040C900087150800BC
:084000000500030002000600A8
:02400E00CC33B1
:10420000010003000300030003000200020002009B
:104210000200000000000000000003000300FF0097
:10422000810000000000000000000000000000000D
:104230000000C000C000C000C000C000C000FF00FF
:10424000FF00C300F300CF00FF00C300F300CF0066
:10425000FF00C300F300CF00FF00C300F300FF0026
:104260000000FF00FF00FF00FF00FF00FF00FF0055
:10427000FF00FF00FF00FF00FF00FF00FF00FF0046
:10428000FF00FF00FF00FF00FF00FF00FF00FF0036
:10429000FF00FF00FF00FF00FF00FF00FF00FF0026
:1042A000FF00FF00FF00FF00FF00FF00FF00FF0016
:1042B000FF00FF00FF00FF00FF00FF00FF00FF0006
:1042C000FF00FF00FF00FF00FF00FF00FF00FF00F6
:1042D000FF00FF00FF00FF00FF00FF00FF00FF00E6
:1042E000FF00FF00FF00FF00FF00FF00FF00FF00D6
:1042F000FF00FF00FF00FF00FF00FF00FF00AA001B
:00000001FF
